:020000020000FC
:1000000009C0000000003DC000000000000000002A
:10001000000000000FE90DBF0FE501BF07E007BBBF
:1000200008E008BB8CE0992702E003BF02E009BFAB
:100030002CE017EE00270A95F1F71A95D9F72A95C3
:10004000C1F704E0800F8F7000E1B39B800FC19A6D
:1000500056D0C198B49902C07894C19AB499F894D2
:10006000E7CFE01038C0E01038C4E01038C8E01026
:1000700038CCE01039F0E01039F1E01039F2E0103E
:1000800039F3939590FDC29A90FFC29818955BE062
:10009000C09AC29A64E26A95F1F7C098C29862E287
:1000A0006A95F1F75A95A1F756E168E46A95F1F778
:1000B0005A95D9F7089556E1C09AC29A64E26A95B2
:1000C000F1F7C098C29862E26A95F1F75A95A1F7E4
:1000D0005BE068E46A95F1F75A95D9F7089518E05E
:1000E0003327001C10F0E7DF02C0D1DF30951A95EE
:1000F000C1F7332311F4CBDF01C0DDDF08954427BE
:10010000F0E0E2E6E40FE80FC895E9DF43954430FC
:04011000B9F708959E
:00000001FF
